:100000000C9496010C94BE010C94BE010C94BE019C
:100010000C94BE010C94BE010C94BE010C94BE0164
:100020000C94BE010C9437030C94B7230C946922F2
:100030000C94BE010C94BE010C94BE010C94BE0144
:100040000C94540A0C94BE010C94BE010C94BE0195
:100050000C94BE010C94BE010C94BE010C94851A44
:100060000C94BE010C945E1F0C94A11F0C94BE0155
:100070000C94BE010C94BE010C94BE010C94BE0104
:100080000C94BE010C94BE010C94BE010C94BE01F4
:100090000C94BE010C94BE010C94BE010C94BE01E4
:1000A0000C94BE010C94BE010C94BE0104130A13FF
:1000B000101317132513471365138E1B911B841BF5
:1000C000881BB21BB21BB21B951B991B9D1BA31B4C
:1000D000A71BB21BAD1B434C49206E6F7420617689
:1000E00061696C61626C652C2075736520636F6E4D
:1000F000666967757261746F72210000000002000A
:10010000080E0000030401000B00000000000000C6
:100110000000000000000000000408020110408000
:1001200040102040804080080204018040201002DE
:10013000011080102040400404040404030405025C
:100140000202020403020202020606060606060472
:100150000402020204000000002300260029002CF3
:10016000002F0000000000250028002B002E003189
:100170000000000000240027002A002D00300008A5
:100180000B0002020201000904000001020200004B
:1001900005240010010524010101042402060524A0
:1001A0000600010705810310004009040100020A4E
:1001B000000000070502024000000705830240001E
:1001C0000000C18081C112010002020000404123F1
:1001D000368000010102000112010002000000400F
:1001E0004123368000010102000118034100720022
:1001F0006400750069006E006F0020004C004C0028
:1002000043002203410072006400750069006E0023
:100210006F0020004C0065006F006E0061007200EE
:1002200064006F00040309040000000000000000E7
:100230002A2B280000000000000000000000000041
:1002400000000000000000002C9EB4A0A1A2A43475
:10025000A6A7A5AE362D3738271E1F20212223241E
:100260002526B333B62EB7B89F8485868788898ABA
:100270008B8C8D8E8F909192939495969798999A56
:100280009B9C9D2F3130A3AD350405060708090A54
:100290000B0C0D0E0F101112131415161718191A36
:1002A0001B1C1DAFB1B0B500090402000103000022
:1002B00000092101010001226500070584034000B7
:1002C0000105010902A1010901A100850105091922
:1002D000012903150025019503750181029501751A
:1002E00005810305010930093109381581257F751C
:1002F0000895038106C0C005010906A10185020514
:100300000719E029E7150025017501950881029577
:1003100001750881039506750815002565050719FF
:100320000029658100C03F1D8F20532511241FBE69
:10033000CFEFDAE0DEBFCDBF12E0A0E0B1E0E2E552
:10034000FDE402C005900D92AA35B107D9F715E07A
:10035000AAE5B2E001C01D92A831B107E1F713E0B0
:10036000CCE2D3E004C02297FE010E941C26C632D4
:10037000D107C9F70E94CB200C94A7260C9400004B
:1003800080910008909101088737974709F0A89558
:100390000895DC01ED91FC910190F081E02D09952B
:1003A000089520919C0330919D03382748E0C901AE
:1003B000880F991F37FF06C09C0151E2252750E1A5
:1003C000352701C09C01415091F730939D03209344
:1003D0009C03089588E380939E0380E092ECA1E063
:1003E000B0E080939F039093A003A093A103B093E8
:1003F000A20387E08093AB0380EC9AECA9E8B6E314
:100400008093A3039093A403A093A503B093A603A2
:1004100085E08093AC038DEE9EEFADEABEED809358
:10042000A7039093A803A093A903B093AA03EDEAAE
:10043000F3E080E090E0863028F4DC01AC5DBD4F55
:100440002C9101C020E0219301968831910599F704
:1004500082E08093C5038AE08093C603089580EC10
:1004600097EFAAEBB7E38093E3039093E403A093A1
:10047000E503B093E60380E090E0A0E0B0E5809370
:10048000E7039093E803A093E903B093EA03EBEE4C
:10049000F3E080E081938F5F8031E1F70895A0E081
:1004A000B0E0E5E5F2E00C94E525D82F0E94DB1AD8
:1004B0006115710581059105C9F30E948826109286
:1004C000A7031092A8031092A9031092AA03C4E0F4
:1004D000812C912C54018A94C090A703D090A8033A
:1004E000E090A903F090AA03FE2CED2CDC2CCC2488
:1004F0000E948326A50194010E94C4256C0D7D1DD8
:100500008E1D9F1D6093A7037093A8038093A9037A
:100510009093AA03C15001F7DD2309F450C00DEAFE
:1005200013E0E801A12CB12C62E3C62ED12CE12C02
:10053000F12C8881882309F442C0B39419F40E94F5
:10054000EA013DC00E948326A70196010E94C425AE
:10055000E1E0E60FADEAB3E08A2F801B8A1520F4B4
:100560008D918E13F9CFE9CF2091AC0330E0A0E15B
:10057000B7E20E945C259B01AC01AE2FB0E00E9467
:100580006B254090A3035090A4036090A503709046
:10059000A603640D751D861D971D4090E3035090C2
:1005A000E4036090E5037090E6034616570668067C
:1005B000790618F2E993A39488E1A812BACFCDB7CF
:1005C000DEB7E0E10C94012680919B03813019F4A1
:1005D00082E080939B0380919B03833019F484E035
:1005E00080939B03089588E08093C10061E08AE0D6
:1005F0000E94B31B60E08AE00E94EC1B0895009704
:10060000C9F09C0140E050E068E478EE81E090E0C1
:100610000E94C4252F3F31054105510529F020F0E6
:100620002FEF30E040E050E02093D1008091C000F7
:10063000806103C08091C0008F7E8093C0000895C8
:10064000219A229A239860E08BE00E94B31B61E01C
:100650008CE00E94B31B0895EBE6F0E08081806897
:100660008083E8E6F0E080818160808308951F92B6
:100670000F920FB60F9211242F933F934F935F93D6
:100680006F937F938F939F93AF93BF93EF93FF935A
:100690001F9B0E94E402FF91EF91BF91AF919F9148
:1006A0008F917F916F915F914F913F912F910F901B
:1006B0000FBE0F901F901895A1E0B0E0E2E6F3E0C6
:1006C0000C94F2251FB791E090939A03F8948983D4
:1006D0000E94C00198E1909360008981809360003E
:1006E00081110E94C0011FBF2196E3E00C940E26E9
:1006F0008F929F92AF92BF92CF92DF92EF92FF9232
:10070000CF93FC01C0A5EC2FE770F0E0E45EFD4F55
:10071000A081B0E0C7FF03C024E130E002C02FE0B9
:1007200030E0FC0197A183E1989FF0011124E25C85
:10073000FE4F80809180A280B380A20FB31F20E47F
:100740003FE14DE750E00E947625A50194010E940B
:10075000A2258C2F887149F469017A01E0EDCE0E53
:10076000E7E0DE1EE11CF11C1BC0C7FF05C060E412
:100770007AE88CE29EE004C060E07EEE8AEB9BE0CB
:1007800069017A01F8EBCF0EFBE0DF1EE11CF11CE2
:10079000A50194010E94A225C20ED31EE41EF51EDF
:1007A000C701B60169517C4F8F4F9F4F28EE33E050
:1007B00040E050E00E94A225A8EEB3E00E946B2525
:1007C000CF91FF90EF90DF90CF90BF90AF909F9030
:1007D0008F9008958F3F910551F048F0811522E0E8
:1007E000920738F08115934030F482E0089580E05C
:1007F000089581E0089583E00895A0E0B0E0E3E08B
:10080000F4E00C94EE25EB018A01B82FB695A0E038
:1008100028813981F80120832A813B8121832C8121
:100820003D8122832E813F812383688179814A81A2
:100830005B812C813D81EE81FF819F2F9295990FE5
:10084000990F907C272F2370922B252F2370220F36
:10085000220F922B232F23702295207F922BF801B9
:1008600094830B5F1F4F2896AF5FBA1788F680FFFF
:1008700024C0888199810E94EA03D82E8A819B81B5
:100880000E94EA03E82E8C819D810E94EA03F82EE3
:100890008E819F810E94EA03F0E4DF9EA001112473
:1008A00090E1E99E90011124242B282BE4E0FE9E88
:1008B000B0011124262BF8012083CDB7DEB7E7E085
:1008C0000C940A26803223E0920708F1883E23E048
:1008D000920740F48F519340E4E096958795EA950E
:1008E000E1F70895803D27E0920718F48C5D93406E
:1008F0000895883928E0920768F4885C974074E08E
:10090000969587957A95E1F78D509C4F089580E0F4
:1009100090E008958FEF93E008958C30910540F4B6
:10092000A4E0880F991FAA95E1F7885D9C4F089570
:10093000843F23E0920718F484529C4F0895811558
:1009400024E0920740F48657934FF4E0880F991FF4
:10095000FA95E1F7089580E998E008959C013695AD
:10096000279525753575821B930B9C012373337373
:10097000969587959695879583739373820F931FAA
:100980009C0154E0369527955A95E1F7280F391FB9
:100990002F703F7041E051E0249FC001259F900DD2
:1009A000349F900D1124892F08952998882319F0D8
:1009B00000002A9A02C000002A980000299A00002C
:1009C0000895299A000083B12998000083FB8827A5
:1009D00080F90895CF93DF93D82F5E9A29985E9877
:1009E000C8E08D2F80780E94D504DD0FC150C9F773
:1009F0002998DF91CF9108958F770E94EA04089596
:100A0000CF93DF93D82FC8E08D2F80780E94D50434
:100A1000DD0FC150C9F72998DF91CF910895CF9389
:100A2000DF932998C8E080E0D82FDD0F0E94E10411
:100A30008D0FC150C9F7DF91CF9108950E94FC043A
:100A40000E940F055E9A0895A1E0B0E0EAE2F5E0A9
:100A50000C94F325806869830E94EA046981862FDB
:100A60000E9400055E9A2196E2E00C940F26CF9337
:100A7000C091A703C827E82FF0E0E256FC4F678536
:100A800089E70E9424056C2F8DE30E9424056C2FBA
:100A900082E40E942405CF91089586E20E941E05FB
:100AA0000895CF93DF93EC016C818CE10E942405C3
:100AB0006D818DE10E9424056E818EE10E942405E6
:100AC0006F8180E20E942405688581E20E942405EE
:100AD000698582E20E9424056A8583E20E942405DA
:100AE0006B8584E20E9424056C8585E20E942405C2
:100AF0006D858AE20E9424056E858EE60E9424059B
:100B00006F858FE60E942405688980E70E9424058E
:100B1000698981E70E9424056A8982E70E94240589
:100B2000DF91CF910895CF92DF92EF92FF92CF9312
:100B3000DF936B017C01C11488E3D8068CE9E806D9
:100B40008CE1F80628F5C701B60120E836E948E946
:100B500050E00E94A225E901689760E879E687E6FF
:100B60009FEF0E947E256C0D7D1D8E1D9F1DF2E066
:100B7000660F771F881F991FFA95D1F721E732E09A
:100B800040E050E00E94A225F22EE32E80E421C036
:100B9000C701B60120E03DE241E351E00E94A225F9
:100BA000E901689760E073ED8EEC9EEF0E947E2570
:100BB0006C0D7D1D8E1D9F1D660F771F881F991F51
:100BC00021E732E040E050E00E94A225F22EE32E21
:100BD00080E66C2F6F71680F85E70E9424056E2DEB
:100BE00086E70E9424056F2D87E70E942405DF9188
:100BF000CF91FF90EF90DF90CF900895682F8DE612
:100C00000E94240508958F929F92AF92BF92CF9237
:100C1000DF92EF92FF92CF93DF93D82F83E00E9471
:100C20001E058093990384E00E941E05809398031B
:100C300060E086E00E94240561E087E00E942405D0
:100C40006FE789E00E94240565E08AE00E942405A0
:100C500065E18BE00E94240562E18CE00E9424059E
:100C60006DEF8DE00E94240560E08EE00E94240577
:100C7000DD2319F08BE291E008C02091C50333E138
:100C8000239FC0011124825C9E4F0E9451056CE895
:100C900080E30E9424056FE082E30E94240562E461
:100CA00083E30E9424058091C60387FF02C064E1AC
:100CB00001C06AE084E30E9424056AE285E30E94A1
:100CC00024056DE286E30E94240564ED87E30E941B
:100CD000240560E088E30E94240560E089E30E9427
:100CE0002405D11109C0C090A703D090A803E090BB
:100CF000A903F090AA0307C0C5E9CC2EC1ECDC2EF5
:100D0000ED2CCEEDFC2ECAE38F2C9924AA24BB2413
:100D1000682D8C2F0E942405682D85E08C0F0E9481
:100D20002405FE2CED2CDC2CCC24CF5FCE3361F7D8
:100D30006FEF83E40E9424056FEF84E40E94240592
:100D40006FEF85E40E9424056FEF86E40E9424057E
:100D5000DD2311F066E002C06091AB038DE60E94D6
:100D6000240560E089E70E9424056091AC038AE7CE
:100D70000E94240560E083E70E94240560E084E788
:100D80000E942405D11109C06091A3037091A403AE
:100D90008091A5039091A60304C060EC7AEC89E8E9
:100DA00096E30E949305DF91CF91FF90EF90DF9043
:100DB000CF90BF90AF909F908F90089561E087E0B3
:100DC0000E94240564E28EE70E94240563E088E027
:100DD0000E94240560E088E00E94240565E087E029
:100DE0000E94240562E085E00E94240583E00E94C1
:100DF0001E058093990384E00E941E05809398034A
:100E0000089583E00E941E058093990384E00E9468
:100E10001E058093980361E087E00E9424056AE044
:100E200070E080E090E00E94FE1A0E94DE06000062
:100E30000895CF92DF92FF920F931F93CF93DF938A
:100E40001F92CDB7DEB7082F162F8EE399830E942D
:100E50002405F02EC02E9981D92E8C2D8F19811743
:100E600038F4F60161916F018FE70E942405F5CFF8
:100E700064E085E00E94240583E00E941E058093C3
:100E8000990384E00E941E05809398030E94DB1A58
:100E900060939403709395038093960390939703C4
:100EA00069E087E00E94240581E080939B030F9016
:100EB000DF91CF911F910F91FF90DF90CF90089518
:100EC0000F931F930E94190780919B03813099F41F
:100ED0000E94DB1A009194031091950320919603D0
:100EE00030919703601B710B820B930B603A76482D
:100EF0008140910548F380919B03813031F467EA8A
:100F000071E086E094E00E94E31D1F910F91089527
:100F10000F931F9380919B03823021F410929B03C7
:100F200081E020C080919B038130D9F40E94DB1ABC
:100F300000919403109195032091960330919703AB
:100F4000601B710B820B930B613A764881409105CF
:100F500040F061E087E00E94240510929B0382E04C
:100F600001C080E01F910F910895CF93DF93EC01B2
:100F70004AE050E06D2F70E086E094E00E94A81EE9
:100F80006EE286E094E00E94B51DBE0184E0769595
:100F900067958A95E1F76F7077274AE050E086E021
:100FA00094E00E94A81E6EE286E094E00E94B51DC7
:100FB000BE016F7077274AE050E086E094E00E941F
:100FC000A81EDF91CF910895D82FC0E0CD1780F4EF
:100FD0005F9A64E670E080E090E00E94FE1A5F98FD
:100FE00064E670E080E090E00E94FE1ACF5FEECFF2
:100FF0006CE271E080E090E00E94FE1AE6CF0F9371
:101000001F93CF93DF93EC01062F15E0115051F0A1
:10101000CE010E949126081741F0602FCE010E9458
:101020009926F4CF82E00E94E407DF91CF911F91CF
:101030000F910895A0E0B0E0E0E2F8E00C94E5251F
:10104000482E562EC0E0D0E0612C712CE12CF12C02
:1010500000E010E041100CC06090FC0386E4689E44
:101060003001112459E1E52EF12C02EE13E01EC0EF
:1010700091E049120FC06090FC03E6E46E9E3001DF
:101080001124FBE16F0E711C49E2E42EF12C0EE9F4
:1010900013E00CC082E0481209C028E1622E7724D8
:1010A0007394EE24E394F12C0BEF13E043018C0EC8
:1010B0009D1E10929D0310929C033401A62CA8182B
:1010C000B12CC30101966C01AE14BF04A8F4A00EAC
:1010D000B11E511006C0C3010E949126F501808304
:1010E00005C0F5016081C3010E94FF07F501808101
:1010F0000E94D1013601E2CFC301511018C0C301D3
:101100000E949126B82EC6010E9491262B2D30E018
:10111000322F2227282B80919C0390919D038217C8
:10112000930779F4C0E0D0E05524539493CF36016F
:1011300060919D030E94FF0760919C03C6010E947D
:10114000FF07C05EDE4FC13E92E0D90708F482CFB0
:10115000852DCDB7DEB7E0E10C94012661E082E099
:101160000E941A08089560E082E00E941A088091A7
:10117000FB03853020F01092FB030E94AE088091A3
:10118000FB038093FC03089561E080E00E941A084D
:1011900061E081E00E941A08089560E080E00E940A
:1011A0001A08882351F060E081E00E941A08882321
:1011B00021F080919E03883349F00E942F020E9403
:1011C000EA0181E00E944F020E94C4080895CF9373
:1011D000C82F0E94DB1A60935803709359038093C1
:1011E0005A0390935B03C0936D03CC2329F040E036
:1011F00051EE60E070E004C040E855E260E070E06D
:1012000088E594E00E940E20CF91089590915C03B0
:10121000492F4F7050E0BA016F5F7F4F292F30E0A8
:10122000E4E035952795EA95E1F76217730759F0E1
:10123000FA01E35AFC4F808381E0890F8F70907F21
:10124000892B80935C0308956EE770E088E594E055
:101250000E94C9010895A3E1B1E0E1E3F9E00C9433
:10126000E625EDEAF3E0712C8191882321F0739457
:1012700028E17212F9CF63EB71E086E094E00E94FE
:10128000E31D4AE050E0672D86E094E00E94AF1E27
:1012900080E00E9403060E94DE068E010E5F1F4F53
:1012A000C12CD12C7601C39466246A945C2C0E94D4
:1012B000CF1A4B015C012091AC0330E0A0E1B7E212
:1012C0000E945C259B01AC01C701B6010E947E25EE
:1012D0002091A3033091A4034091A5035091A6034C
:1012E000620F731F841F951F2091E3033091E40365
:1012F0004091E5035091E603261737074807590741
:1013000018F4F801608225C08C2D0E94370561E039
:1013100070E080E090E00E94FE1AF80110820E94C6
:10132000CF1A681979098A099B09643F71408105C0
:10133000910540F40E944D05F8019081981778F7C7
:101340008083EDCF50FE03C046985F9A02C0469A54
:101350005F982FEFC21AD20AE20AF20A0F5F1F4FFC
:101360008FEFC816D104E104F10409F09FCFCE013C
:101370009395FC01D82E7FEF68EC2E2F281B2715A4
:1013800010F051E056C0DE01129651E02FEF41E01F
:101390003D91321710F0322F01C0452F5F5F5F3F44
:1013A00011F0232FF5CF4193242F30E0A1E0B0E0DE
:1013B000AC0FBD1FA20FB31F5C93413079F0DE016B
:1013C000A20FB31F5C93423049F0AFEFBFEFAC0FF9
:1013D000BD1FA20FB31F6C934E3F78F6A2E0B0E0A2
:1013E000AC0FBD1FA20FB31F7C934D3F30F6A3E09F
:1013F000B0E0AC0FBD1FA20FB31F6C93BECF452F43
:10140000242F30E0FC01E20FF31F6081AFEFB0E06A
:10141000AC0FBD1FA20FB31F2C91621748F44150AF
:10142000DC01A40FB11D2C9120836C934111E8CFF6
:101430005F5F571520F3372D369520E0231770F4A2
:10144000DC01A20FB11D4C91522F530FFC01E50F8F
:10145000F11D50815C9340832E5FF0CFFDEAEF2EAB
:10146000F3E0FF2E8C01802F8D19871598F4F80179
:10147000C1908F014AE050E06C2D86E094E00E941C
:10148000A01E6CE286E094E00E94B51DF701C192B7
:101490007F01E9CF86E094E00E94BD1D81E0CD5E32
:1014A000DE4FEFE00C9402261F920F920FB60F92C0
:1014B00011241F932F933F934F935F936F937F93C9
:1014C0008F939F93AF93BF93CF93DF93EF93FF934C
:1014D000C0918600D09187008091170390911803E6
:1014E00020913903211155C09E01281B390B809191
:1014F000E7039091E803A091E903B091EA0385FD29
:1015000002C036952795253C49E03407B8F1409153
:101510000A0150E060E070E02CE1B695A795979540
:1015200087952A95D1F70097A105B10521F481E0AF
:1015300090E0A0E0B0E084179507A607B707D8F4BD
:1015400080910A018F3FB9F040E080910A0148176D
:1015500080F4842F90E0880F991FFC01E75EFC4F18
:1015600020813181FC01E55FFE4F318320834F5F95
:10157000ECCF10923A0310920A010BC02D3B82E08F
:10158000380720F080910A018031D8F08FEF8093E6
:101590000A01D0931803C0931703FF91EF91DF91D5
:1015A000CF91BF91AF919F918F917F916F915F91FB
:1015B0004F913F912F911F910F900FBE0F901F9051
:1015C000189510910A0181E0810F80930A01C901E9
:1015D0000E946204E12FF0E0EE0FFF1FE75EFC4F78
:1015E00091838083D6CF83E0809380008AE98093C3
:1015F00081008091E70386FD05C0809181008064B1
:10160000809381008FEF9FEF9093890080938800F3
:1016100080916F00806280936F000895CF93DF9375
:101620000E94B3088091FC03843039F582E00E9467
:101630001F1CC1E0D0E0892B11F4C0E0D0E083E0B2
:101640000E941F1C892B19F082E090E002C080E00C
:1016500090E08C2B9D2B8230910539F083309105E1
:1016600039F0019739F481E006C01092FC0305C0FF
:1016700082E001C083E08093FC03DF91CF91089565
:101680006F3018F086958058089589E0689F802D06
:1016900011240895A0E0B0E0E0E5FBE00C94ED2516
:1016A000C82F0E94DB1A0091C8021091C902209134
:1016B000CA023091CB026B017C01C01AD10AE20A46
:1016C000F30A9701860149E8C41643E1D406E10410
:1016D000F10410F01092CC026093C8027093C9021A
:1016E0008093CA029093CB02209139038FEF820F2F
:1016F0008230D8F5E091CC02EE2309F44EC1E130FE
:1017000011F482E0B8C1E03108F034C181E08E0FFD
:101710008093CC02F0E0E75EFC4FC083803109F09B
:10172000ACC1EBE1F3E0213029F4A181A695A695A7
:10173000808108C080819181A92FA695A695A69544
:1017400096958795A03148F4B0E090E0AA0FBB1FB2
:10175000A55FBE4F11969C938E9310923A033296DA
:1017600083E0E932F807F9F688C1233009F005C1B2
:10177000E091CC02E11104C0CF3009F07EC10DC16F
:10178000E83148F481E08E0F8093CC02F0E0E85E0F
:10179000FC4FC08372C1E83109F0ECC0C111EAC04E
:1017A00040E050E0ABE0CA01B3E0880F991FBA9562
:1017B000E1F7A49F9001A59F300D1124F901E75E88
:1017C000FC4F6081E1817E2F777075956795FC01F4
:1017D000EE0FFF1FE55FFE4F71836083F901E65E48
:1017E000FC4FB081B695B695B695E181FE2FF29586
:1017F000FF0FF07E6F2F6B2BE695E695E6957E2F1B
:10180000777075956795FC01EE0FFF1FE35FFE4F44
:1018100071836083F901E55EFC4FB081B295B695A6
:10182000B695B370C181DC2FDD0FDD0F6D2F6B2BF3
:10183000C295C695C695C370E281E170EE0FEE0FBA
:101840007E2F7C2B75956795FC01EE0FFF1FE15FE6
:10185000FE4F71836083F901E35EFC4FB081B69562
:10186000E181FE2FF795FF27F7956F2F6B2BE695FC
:101870007E2F777075956795FC01EE0FFF1FEF5E69
:10188000FE4F71836083F901E25EFC4FB081B29537
:10189000BF70E181FE2FF295F07F6F2F6B2BE295E9
:1018A000EF707E2F777075956795FC01EE0FFF1F27
:1018B000ED5EFE4F71836083F901E15EFC4FB08104
:1018C000BB1FBB27BB1FC181DC2FDD0F6D2F6B2B17
:1018D000CC1FCC27CC1FE281E370EE0F7E2F7C2B38
:1018E00075956795FC01EE0FFF1FEB5EFE4F718350
:1018F0006083F901EF5DFC4FB081B695B695E1814B
:10190000FE2FF295FF0FFF0FF07C6F2F6B2BE695EC
:10191000E6957E2F777075956795FC01EE0FFF1F9A
:10192000E95EFE4F71836083F901EE5DFC4F20811B
:101930002295269527703181E32FEE0FEE0FEE0FE3
:101940006E2F622B732F72957695777075956795CC
:10195000FC01EE0FFF1FE75EFE4F718360834F5F58
:101960005F4F4230510509F01ECF80912F0383FF56
:1019700010923A031092CC0280C0243009F07DC04E
:101980006091CC0261110BC0C83AB1F410929D0372
:1019900010929C0388EA0E94D10181E06CC0613002
:1019A00019F4C093C70204C0623031F4C093C60278
:1019B0008C2F0E94D1015AC0E091C6022E2F30E038
:1019C000220F331F462F50E0C90102968417950756
:1019D0003CF0633268F7FA01EA5EFC4FC083E8CF5F
:1019E0002D5F3F4F8C2F90E060919C0370919D0381
:1019F0004217530749F4982F8827862797279093F3
:101A00009D0380939C0332C06817790769F5809124
:101A1000C702813049F5E13118F080E18093C602B8
:101A2000F090C602CAE1D3E000E010E00F15D0F458
:101A3000FE013197808190E0982F88272881822BA2
:101A400063E0969587956A95E1F70E946204F80134
:101A5000EE0FFF1FE55FFE4F918380830F5F1F4FE7
:101A60002296E4CF10923A031092CC028091CC02DD
:101A7000882319F08F5F8093CC02CDB7DEB7E8E002
:101A80000C940926CF93DF93E82FF0E0EE51FC4F42
:101A9000E185E03150F4F894F0E0EE0FFF1FE55FD0
:101AA000FE4F8081918178945FC08EE08E0F8B30E5
:101AB00058F4F0E0E25FF10924E62E9FC0012F9F69
:101AC000900D11240C9650C0E03F09F448C038F442
:101AD000E131A1F0E231A1F0E03139F409C0ED3F8C
:101AE000C1F1EE3FC9F1E13F89F180E092E03CC0F5
:101AF00082E00E941F1C892B19F134C083E0F9CFCA
:101B000082E00E941F1CC1E0D0E0892B11F4C0E0EC
:101B1000D0E083E00E941F1C892B19F082E090E046
:101B200002C080E090E08C2B9D2B8230910541F02B
:101B30008330910541F00197A9F086EA92E014C044
:101B40008CE090E011C089E591E00EC086E090E065
:101B50000BC08AEF93E008C08FEF93E005C080E0F0
:101B600090E002C084EF93E0DF91CF910895A2E26C
:101B7000B0E0EDEBFDE00C94E3259E012F5F3F4FBD
:101B800080E1D9011D928A95E9F761EE71E086E066
:101B900094E029A33AA30E94E31D0E9401071D8A35
:101BA0001E8A1F8A188E312C212C00E0812C912C4A
:101BB000540170EC472E7DE9572E78E5672E75E3CA
:101BC000772EE0E5CE2EE3ECDE2EE12CF12C84EF37
:101BD00091E0A0E0B0E08D8F9E8FAF8FB8A380EC36
:101BE00097EFAAEBB7E3898F9A8FAB8FBC8F80EC0E
:101BF0009DE9A8E5B5E3898B9A8BAB8BBC8B86E01E
:101C000094E00E94481C892B09F4E1C086E094E02E
:101C10000E946C1C9C0133272C32310509F442C010
:101C2000ACF42332310509F0ABC019821A821B8251
:101C30001C821D821E821F82188619861A861B86A8
:101C40001C861D861E861F86188A60C024343105B6
:101C500029F02335310509F4B2C092C064E486E06E
:101C600094E00E94B51D2AE030E040EC5DE968E5B3
:101C700075E386E094E00E94431E6CE286E094E007
:101C80000E94B51D2AE030E040EC57EF6AEB77E3A5
:101C900086E094E00E94431E6CE286E094E00E949D
:101CA000F51DADCF0F5F043009F0A9CF29813A812E
:101CB0004B815C81A8EEB3E00E946B25698B7A8B27
:101CC0008B8B9C8B2D813E814F8158850E946B258B
:101CD000698F7A8F8B8F9C8F29853A854B855C85A0
:101CE0002D8F3E8F4F8F58A32D853E854F85588968
:101CF0000E946B256B017C0160323EE47307810515
:101D0000910530F462E38CE10E94240500E077CF76
:101D1000603345E774078105910510F462E2F3CF63
:101D200060345CE975078105910510F466E2EBCF3C
:101D300080E5C81683ECD806E104F10410F462E1F2
:101D4000E2CF90E6C9169AEED906E104F10410F448
:101D500065E1D9CFA0E7CA16A1E1DA06A1E0EA065B
:101D6000F10410F461E0CFCFB0EACB16B6E8DB06A1
:101D7000B1E0EB06F10410F463E0C5CF65E0C3CF3A
:101D800010ED180F1A3008F03ACFE1E0F0E0EC0F58
:101D9000FD1F24E0029FE00DF11D112420813181FF
:101DA00042815381AAE0B0E00E946B25610F711D52
:101DB000811D911D608371838283938320CF498825
:101DC0005A886B887C88812C912C540118CF8114FF
:101DD0009104A104B10489F4C301B2010E949305E6
:101DE00061E070E080E090E00E94FE1A1D8A1E8A89
:101DF0001F8A188E312C22242A948D8D9E8DAF8DB2
:101E0000B8A188169906AA06BB06D0F40E944D0513
:101E10002D893E894F89588D280F311D411D511D37
:101E20002D8B3E8B4F8B588F381608F4382E821529
:101E300008F4282E3FEF831A930AA30AB30A56C068
:101E4000C301B20128EE33E040E050E00E94A22539
:101E5000BA01A9012AE030E086E094E00E94911ED8
:101E60006CE286E094E00E94B51D4AE050E0632DEC
:101E700086E094E00E94A01E6CE286E094E00E945E
:101E8000B51D6D897E898F89988DA50194010E9469
:101E9000A225BA01A9012AE030E086E094E00E9480
:101EA000911E6CE286E094E00E94B51D4AE050E08D
:101EB000622D86E094E00E94A01E6CE286E094E031
:101EC0000E94F51D4C0C5D1C6E1C7F1C898D9A8D2B
:101ED000AB8DBC8D84159505A605B70520F4498802
:101EE0005A886B887C88812C912C540129893A89E5
:101EF0004B895C89283E33404105510509F07FCE6E
:101F0000A296E2E10C94FF25ACE1B0E0EAE8FFE044
:101F10000C94ED250E94DB1A6B017C0181E00E948C
:101F2000030614E703E0198361E0CE0101960E94E5
:101F3000600700939B030E94DE066AEF70E080E07A
:101F400090E00E94FE1A80919B03833089F486E022
:101F500094E00E94481C892B59F40E94DB1A6C19EA
:101F60007D098E099F096038734C894C9140D8F2E5
:101F700080919B03833009F44FC08FE70E94FC04DB
:101F80000E940F058983843511F083E05CC00E94B4
:101F90000F0510926E0380936F030E940F0520912E
:101FA0006E0330916F03280F311D30936F03209320
:101FB0006E030E940F05809370030E940F058093AB
:101FC0007103813110F7F12C0F2D10E08091710316
:101FD00090E0880F991F0817190740F40E940F0519
:101FE000F801EE58FC4F8083F394EECF80E78983AD
:101FF00061E0CE0101960E94600783E080939B031D
:102000000E94DE0662E370E080E090E00E94FE1A2B
:1020100080919B03833011F482E015C08FE70E940A
:10202000FC040E940F058983803509F0AECF07ECD0
:1020300013E00E940F05F80181938F01F3E0023E47
:102040001F07B9F781E06C96E8E00C940926CF935E
:10205000C82F682F86E094E00E94B91C90919203EB
:102060009C2790939203CF910895A1E0B0E0EBE319
:10207000F0E10C94F32599830E9427109981892F10
:102080000E9427102196E2E00C940F261F93CF9315
:10209000DF93182FEB011092920365EB86E094E03A
:1020A0000E94B91C62E686E094E00E94B91C812F70
:1020B0000E942710CE010E943510DF91CF911F9111
:1020C00008956091920386E094E00E94B91C0895FF
:1020D000A1E2B0E0EEE6F0E10C94EF257B018A018D
:1020E0008C3009F453C108F040C0863009F4BCC0FC
:1020F00018F5833009F491C070F4813009F472C08E
:10210000823009F048C26BE170E082E00E94461024
:1021100007EC13E078C0843009F487C0853009F0FB
:102120003AC26091710370E0660F771F85E00E94EC
:10213000461002E713E086C0893009F4A7C070F4A6
:10214000873009F49BC0883009F025C261E070E057
:1021500088E00E9446108091FC0323C28A3009F473
:10216000CAC08B3009F4F2C016C28A3609F475C1B0
:10217000D8F4873609F43AC138F4853609F40EC12B
:10218000863609F41FC107C2883609F437C189367B
:1021900009F001C261E070E089E60E9446100E94E9
:1021A000EA010E942F02F5C18D3609F4D4C138F43A
:1021B0008B3609F491C18C3609F49AC1ECC18E3684
:1021C00009F4DCC1873C09F0E6C161E070E087EC0E
:1021D0000E94461081E00E9427100E946110109218
:1021E0009303E3C169E270E081E00E9446100EE9CA
:1021F00013E0F80181918F010E942710F3E0073C62
:102200001F07B9F7D0C1F80181918F010E942710F3
:10221000F3E0023E1F07B9F7C6C161E070E083E05A
:102220000E9446100E94840FBCC161E070E084E00F
:102230000E94461081E00E9427100E9461100E94B7
:10224000B70DB3C18091710390E0880F991F980179
:10225000225733402817390708F0A5C1F8018191AA
:102260008F010E942710EECF62E070E086E00E94AE
:10227000461085E893E00E94351095C161E070E05A
:1022800087E00E944610809170038BC186E68983A7
:1022900061E0CE0101960E9460070E94DE0683E0A5
:1022A00080939B0368EC70E080E090E00E94FE1A4F
:1022B00080919B038430D9F48FE70E94FC040E9434
:1022C0000F058983863469F460E270E089E00E943A
:1022D000461010E20E940F050E9427101150D1F7FE
:1022E00062C161E070E089E00E94461052C161E085
:1022F00070E089E053C169E170E08AE00E94461015
:1023000082E08093E20320919A038091E703909109
:10231000E803A091E903B091EA03222311F0806859
:1023200001C08F778093E7039093E803A093E903BC
:10233000B093EA0302EE13E0F80181918F010E944D
:102340002710F3E00B3F1F07B9F72DC161E270E0E2
:102350008BE00E94461080913A038F3F39F08091C4
:102360003A0391E0980F90933A0302C080913A03A8
:102370000E94271010E0812F0E94420D0E948D04C0
:102380000E9435101F5F1031B1F70DC161E070E0A0
:102390008CE00E9446108091FB0303C161E070E075
:1023A00085E60E94461089E2E816F10409F0F8C0BB
:1023B000D801EEE9F3E08D91819383E0E73CF807E3
:1023C000D1F7E7C061E070E086E60E944610EBE1DD
:1023D000EE16F10409F0E4C0D801E7ECF3E08D91CA
:1023E000819383E0E23EF807D1F7D3C061E070E06B
:1023F00087E60E9446100E94C408CBC061E070E0EE
:1024000088E60E94461085E789838BE1E7ECF3E0DC
:10241000DE01129601900D928A95E1F76CE1CE01F2
:1024200001960E9460070E94DE0683E080939B0372
:1024300060E273E080E090E00E94FE1A80919B03CE
:10244000843009F0ADC08FE70E94FC040E940F05A4
:102450008983853509F0A4C09CC061E070E08AE6FC
:102460000E94461089E6898361E0CE0101960E94B0
:1024700060070E94DE0683E080939B0360E273E0C6
:1024800080E090E00E94FE1A80919B03843009F066
:1024900087C08FE70E94FC040E940F0589838E018C
:1024A0000E5F1F4F7E01EDE1EE0EF11C0E940F0545
:1024B000F80181938F01EE15FF05C1F78BE1FE0155
:1024C0003296A7ECB3E001900D928A95E1F78981ED
:1024D000893409F065C05DC061E070E08BE60E9460
:1024E0004610F80180818093FC030E94CD0851C002
:1024F00061E070E08CE60E944610F0E2EF16F10415
:1025000061F487E6898380E2F801DE01129601908A
:102510000D928A95E1F761E203C087E4898361E067
:10252000CE0101960E9460070E94DE0683E0809340
:102530009B036CE474E080E090E00E94FE1A8091BE
:102540009B03843069F58FE70E94FC040E940F050D
:10255000873431F51EC061E070E08DE60E944610C0
:1025600089E1E816F104E1F4D801E2EEF3E08D919F
:10257000819383E0EB3FF807D1F70BC061E070E097
:102580008EE60E944610F80180818093FB030E9432
:10259000AE0881E006C061E070E08AEC0E9446105F
:1025A00080E00E9427100E946110A196E6E00C9442
:1025B0000B26A0E0B0E0EFEDF2E10C94ED25CAE5CA
:1025C000D2E014E606E035E0F32E44E0E42E53E0DA
:1025D000D52E62E0C62E86E094E00E94481C892B2E
:1025E00009F49BC086E094E00E946C1C282F809325
:1025F000C5024091C40250E04730510560F7FA012E
:10260000EA5AFF4F0C941A26853B29F781E0809304
:10261000C402E1CF823609F07DC0C092C402DBCF94
:102620008093C3028093C202D092C402D4CF9C0193
:1026300033273093C1022093C0029091C2029827A1
:102640009093C202E092C402C6CF382F2227409155
:10265000C0025091C102242B352B3093C10220932C
:10266000C0029091C20298279093C202F092C402D5
:102670002536310508F4AFCF61E070E08CEC0E94A4
:10268000461081E00E9427100E94611043C02091F3
:10269000BE023091BF02F901E65AFD4F808390914E
:1026A000C20298279093C202C90101969093BF027B
:1026B0008093BE022091C0023091C102821793071D
:1026C00008F489CF0093C40286CF8091C20282139E
:1026D0000BC06091BE027091BF024AE552E080914A
:1026E000C3020E9468100DC062E070E08BEC0E9493
:1026F00046108091C3020E942710809192030E948D
:102700002710FE01812F11928A95E9F71092BF02DE
:102710001092BE021092C4025ECFCDB7DEB7E8E0E1
:102720000C94092681E0809393038091930388237E
:1027300049F086E094E00E94481C892BB1F30E9486
:10274000D912F3CF0895AAE2B0E0E9EAF3E10C94DC
:10275000EB250E94CF1A6B017C0181E00E940306E9
:1027600086E094E00E94481C892B29F086E094E0E2
:102770000E946C1CF5CF5F9811E072E6B72EE9E27B
:10278000AE2E03E00E94CF1A6C197D098E099F09B5
:10279000693C710581059105D0F11123C1F10E94B9
:1027A000CF1A6B017C01469A80ED97E00E94FF02F0
:1027B000B982EEE9F3E0DE0112968A2D01900D92C6
:1027C0008A95E1F76AE2CE0101960E946007469879
:1027D00080E090E00E94FF0200939B030E94DE06CF
:1027E00062E370E080E090E00E94FE1A80919B031B
:1027F000843061F400939B038FE70E94FC040E94E5
:102800000F0511E0823419F410E001C011E082E1FB
:102810000E941F1C892B81F411E00EC05F9A469A1A
:1028200086E094E00E946C1C8D309105A9F05CF468
:102830000A9791F05F98469886E094E00E94481CC1
:10284000892B61F79FCF8332910569F0823491051E
:1028500089F70E949213EECF66ED70E086E094E077
:102860000E94D11DE7CF0E94B70DE4CF8F929F92B7
:10287000AF92BF92CF92DF92EF92FF921F93CF93CE
:10288000DF9382E10E941F1C892B09F089C068EC4C
:1028900070E080E090E00E94FE1A80E090E00E94EC
:1028A000FF020E94CF1A4B015C016B017C0180EC9E
:1028B000C80E82E1D81EE11CF11C0E94CF1A6C15D3
:1028C0007D058E059F0530F482E10E941F1C892B37
:1028D000A1F364C082E10E941F1C892B09F05EC035
:1028E00080ED97E00E94FF020E94CF1A6B017C01ED
:1028F000D0E0C1E088E4880E86E2981EA11CB11CDD
:1029000011E082E10E941F1C892B21F58C149D048B
:10291000AE04BF0430F480ED97E00E94FF02D1E0E6
:10292000F0CF0E94CF1A6C197D098E099F09693C6E
:1029300071058105910528F30E94CF1A6B017C0176
:10294000C12719F080ED97E002C080E090E00E947E
:10295000FF02D7CF80E090E00E94FF02DD23B9F0B4
:102960008091FB0390E0019665E070E00E948E2567
:102970008093FB030E94AE080E940E0B0E94CD08BC
:1029800064EF71E080E090E00E94FE1A09C080E0F0
:102990000E944F020E942B090E94C4080E94A313A8
:1029A000DF91CF911F91FF90EF90DF90CF90BF907C
:1029B000AF909F908F900895CF92DF92EF92FF9209
:1029C00080E00E945C030E94200361E086E00E9498
:1029D000B31B61E085E00E94B31B60E082E10E94CE
:1029E000B31B60E082E00E94B31B61E082E00E94C2
:1029F000EC1B60E083E00E94B31B61E083E00E9477
:102A0000EC1B60E084E00E94B31B61E084E00E9464
:102A1000EC1B0E94F30260E070E086E094E00E940C
:102A20003E1D0E940E0B0E94CD080E94F30A8FEFFC
:102A300080933A030E942C0378940E94CF1A6B0172
:102A40007C0180913A038F3F59F40E94CF1A6C1990
:102A50007D098E099F09603D77408105910588F3C6
:102A600080ED97E00E94FF0261E082E10E94EC1B92
:102A70005F9A86E094E00E94481C892B29F086E04A
:102A800094E00E946C1CF5CF6EEE71E086E094E05D
:102A90000E94B21D85E893E00E94B50765E072E0F0
:102AA00086E094E00E94B21D4AE050E066E070E0EB
:102AB00086E094E00E94791E62E370E080E090E09E
:102AC0000E94FE1A86E094E00E94481C04970CF1D4
:102AD00086E094E00E946C1C82349105D1F486E07B
:102AE00094E00E946C1C8E34910599F486E094E089
:102AF0000E946C1C8434910561F486E094E00E948D
:102B00006C1C819731F480E090E00E94FF020E94EB
:102B1000A31340919F035091A0036091A103709172
:102B2000A203DB01CA010197A109B1090497A1051C
:102B3000B10568F440933903433029F440EA56E87C
:102B400061E070E004C040E052EC61E070E088E5D4
:102B500094E00E940E200E9436145F9880E090E07E
:102B60000E94FF020E94F30A109255038091E7032E
:102B700083FF11C08091B303882351F08091BA0381
:102B8000882331F08091C103882311F087E001C0D0
:102B900085E08093550380E00E94030680915603F0
:102BA0000E9437050E94DE061092CF021092CE02DC
:102BB0001092CD02F12C8091FC038F15B0F062E3EE
:102BC00070E080E090E00E94FE1A80ED97E00E94A5
:102BD000FF0262E370E080E090E00E94FE1A80E075
:102BE00090E00E94FF02F394E6CF8091C60384FF39
:102BF00008C0982F987181E0983109F080E00E9418
:102C0000E7088FE00E945C03FF90EF90DF90CF9089
:102C10000895EF92FF920F931F93CF93DF938C0150
:102C20006EE770E088E594E00E94C901E801F12CAC
:102C3000F0E2EF2E8E0188818D57823048F46DE7E7
:102C400070E088E594E00E94C90188818E25888320
:102C50002196F801608188E594E00E94201FF3949A
:102C6000F9E0FF12E7CF6EE770E088E594E00E949C
:102C7000C901CDB7DEB7E6E00C940B26A9E0B0E0C1
:102C8000E4E4F6E10C94F3259091570391110EC002
:102C90009EEF99838A836B8350E0559547954C83CB
:102CA0002D83198618861F821E822EC040915C03D8
:102CB000842F90E0B4E095958795BA95E1F7242F9D
:102CC0002F7030E08217930719F18DEF89831B82F3
:102CD000FE01349650E0842F90E0A4E0959587950E
:102CE000AA95E1F7242F2F7030E08217930749F05F
:102CF000DC01A35ABC4F8C918193405F5F5F5630DB
:102D000051F740935C035A83CE0101960E94091645
:102D10008091570390E0019666E070E00E948E2556
:102D2000809357032996E2E00C940F26A0E0B0E0D0
:102D3000ECE9F6E10C94EC256C016EE770E088E5B7
:102D400094E00E94C9018601E12CF12CC0E0D0E0A2
:102D500030E2B32EF801608183E8860F823078F488
:102D60006DE770E088E594E00E94C901F801608198
:102D70006B2570E088E594E00E94C90104C088E5F5
:102D800094E00E94201FE114F10459F0F8018081C1
:102D90009E01280F311DC901C92FDD27C80FD91F7A
:102DA000DD273FEFE31AF30A89E0E816F10459F052
:102DB00028E0E216F10421F48C2F8095F60180873B
:102DC0000F5F1F4FC7CFCDB7DEB7E9E00C940826E1
:102DD000A9E0B0E0EEEEF6E10C94F325E82F362FF3
:102DE0008091570390E0019664E270E00E948E2586
:102DF0008093570358E9598350E15A83813089F011
:102E000048F08230B9F08330D9F48B8381EF8C8322
:102E10003D8319C085E08B8381EF8C832F5F2D83E9
:102E200012C08B8381EF8C8384E6489FA00111241C
:102E30005D8309C084E08B8381EF8C83ED8303C0C5
:102E40000E94240904C0CE0101960E94961629967C
:102E5000E2E00C940F26A2E0B0E0E1E3F7E10C948D
:102E6000E825182F762E2A8349830E94DB1A6B01EE
:102E70007C0180916D038090580390905903A0903D
:102E80005A03B0905B032A8149818823C1F0D7019E
:102E9000C60188199909AA09BB094C015D0191EE87
:102EA00089169EE29906A104B10420F1241708F4C2
:102EB000422F202F672D812F0E94E81613C0D701C3
:102EC000C60188199909AA09BB094C015D0191E362
:102ED000891695E79906A104B10460F0672D812F4A
:102EE0000E943E16C0925803D0925903E0925A03B2
:102EF000F0925B032296EDE00C940426A2E2B0E08F
:102F0000E4E8F7E10C94E9258CE00E941E058111AC
:102F10000DC06DE072E086E094E00E94E31D5F9AD0
:102F200080E00E9403060E94DE065F9888E594E038
:102F30000E94C61E892B01F188E594E00E94F31ED1
:102F400090913903992319F00E944A0BEFCF4091D9
:102F5000CE0250E09A012F5F3F4F2F7133276091CF
:102F6000CF0270E02617370709F3FA01E752FD4F49
:102F700080832093CE02DACF80913903811106C07D
:102F800080919B03843009F094C00DC086E094E0EA
:102F90000E94481C892BA1F386E094E00E946C1CDF
:102FA0000E944A0BF3CF0E94DB1A6115710581055F
:102FB000910549F060934703709348038093490358
:102FC00090934A030CC081E090E0A0E0B0E08093D1
:102FD000470390934803A0934903B0934A03809119
:102FE0003D0390913E03816090933E0380933D03A7
:102FF00083E080939B038FE70E94FC0409EF12E0BB
:103000000E940F05F80181938F01F3E002301F0742
:10301000B9F7209102038091F902982F922796FF29
:103020003BC090E4922790930203982F98739833B3
:10303000F1F410E0212F30E08091F902877090E0E8
:10304000821793074CF11F5F2091C603812F90E0F8
:10305000FC01E750FD4F24FF04C080810E94060957
:10306000E9CF608188E594E00E94201FE3CF8F7351
:1030700099F48091FA02809346038091FB02809339
:1030800044038091FC02809343038091FF0290E00F
:1030900090933C0380933B038091CD02813019F4DF
:1030A00082E08093CD028091CD02833011F41092A2
:1030B000CD020E94DB1A6B017C0180913F0390914D
:1030C0004003A0914103B09142030097A105B105CF
:1030D000C9F0A7019601281B390B4A0B5B0BDA01DB
:1030E000C901883B9B40A105B10560F00E944D05D8
:1030F0008093450310923F031092400310924103C6
:103100001092420380914B0390914C03A0914D0388
:10311000B0914E0346015701881A990AAA0ABB0AC0
:103120008EE993E00E94780386169706A806B906F2
:1031300008F4B1C0C0924B03D0924C03E0924D030F
:10314000F0924E030E94C00180913A038830A0F0B3
:103150008091E7039091E803A091E903B091EA031D
:103160005CE1B695A795979587955A95D1F7892BE8
:103170008A2B8B2B09F0B8C180913A038F5F809323
:103180003A038091470390914803A0914903B0917D
:103190004A030097A105B105F1F0C81AD90AEA0A55
:1031A000FB0A8EE993E00E9478036C157D058E057D
:1031B0009F0508F00FC18091E70384FD04C080EDF6
:1031C00097E00E94FF02109247031092480310926A
:1031D000490310924A0390910203907C909302035A
:1031E0005091CE028091CF022091CD02581709F460
:1031F0000EC1223009F00BC1905890930203E09168
:10320000C603E770F0E0E45EFD4F6081693008F0CE
:10321000E6C0615040E04613E4C08093CF0287E3EC
:10322000840F90910203892B809302034093D00274
:1032300083E08093CD02469A1091AB0380915503B1
:10324000811132C18091E70382FD3AC1812F0E9432
:10325000FE05809156030E943705E091C603E77092
:10326000F0E0E45EFD4F608182E093E00E94190788
:103270008091E70382FD2DC1E0915603EF5FE0935B
:103280005603E83109F42DC1F0E0E256FC4F878582
:10329000882309F426C10E948807813069F580914E
:1032A000C603887149F180913D0390913E03880FD8
:1032B000991F90933E0380933D0383E080939B038B
:1032C0000E94DE060E94DB1A60933F037093400366
:1032D0008093410390934203672B682B692B61F421
:1032E00081E090E0A0E0B0E080933F039093400342
:1032F000A0934103B09342038091C60384FF1FC093
:1033000080913D0390913E038E7F0E94AE04182F62
:1033100060913B03809146030E94400B482F612F30
:103320008091450349A30E94400B0091FC03282F84
:1033300049A160914303809144030E942B17469852
:10334000809153038130C1F018F08230B1F1D9C0BF
:1033500082E10E941F1C892B09F0D3C081E0809379
:1033600053030E94CF1A60934F03709350038093CE
:10337000510390935203C5C082E10E941F1C892B08
:1033800031F50E94CF1AC0904F03D0905003E090C7
:103390005103F09052036C197D098E099F09693E13
:1033A00073408105910508F4ACC082E0809353031B
:1033B00080ED97E00E94FF02A4C082E10E941F1CE2
:1033C000892B09F49EC080E090E00E94FF021092D9
:1033D000530397C080E090E00E94FF02FCCE68E0BB
:1033E00019CF851709F419CF4F5F242F30E090E0F3
:1033F000F901EE5FFC4FDC01A752BD4F7C91708359
:10340000F901E053FD4F708301968F7104CF243092
:10341000B1F42091D00281ED92E0A3E0B3E0FC0191
:103420003E2F381B321718F431913D93F9CF87E3C3
:10343000820F90910203892B80930203F9CE809131
:103440005303823051F49160909302035F9A8E018E
:103450000F5F1F4FF12CB80110C05F988091CD0213
:10346000811103C081E08093CD028091CD02833031
:1034700071F784E08093CD02EACF8F2D69A37AA300
:103480000E94420DF801819391938F01F39469A1F9
:103490007AA1F0E1FF12F1CF8091C60343E053E03F
:1034A00087700E94FD03C7CE112309F4CBCE909103
:1034B000540321E0290F209354039813C3CE1DC059
:1034C00082E00E941F1C892B09F0C0CE5F9A17E092
:1034D000BDCE82E00E941F1C892B09F0CDCE5F98E3
:1034E000CBCE10925603D7CE80913A03883009F4A0
:1034F0005F9A89E080933A03CECE10925403115024
:10350000A1CEA296ECE00C9405261F920F920FB666
:103510000F9211242F933F938F939F93AF93BF9359
:103520008091FE039091FF03A0910004B0910104EB
:103530003091FD0323E0230F2D3720F40196A11DC8
:10354000B11D05C026E8230F0296A11DB11D2093D1
:10355000FD038093FE039093FF03A0930004B093B8
:1035600001048091020490910304A0910404B0919D
:1035700005040196A11DB11D8093020490930304DC
:10358000A0930404B0930504BF91AF919F918F91D4
:103590003F912F910F900FBE0F901F9018952FB74E
:1035A000F8946091FE037091FF0380910004909164
:1035B00001042FBF08953FB7F894809102049091C1
:1035C0000304A0910404B091050426B5A89B05C08E
:1035D0002F3F19F00196A11DB11D3FBF6627782F1F
:1035E000892F9A2F620F711D811D911D42E0660F78
:1035F000771F881F991F4A95D1F70895CF92DF92C0
:10360000EF92FF92CF93DF936B017C010E94DB1A54
:10361000EB01C114D104E104F10479F00E94DB1A3A
:103620006C1B7D0B683E7340A0F381E0C81AD10883
:10363000E108F108C851DC4FECCFDF91CF91FF904A
:10364000EF90DF90CF900895789484B5826084BD28
:1036500084B5816084BD85B5826085BD85B5816096
:1036600085BDEEE6F0E0808181608083E1E8F0E0F6
:103670001082808182608083808181608083E0E825
:10368000F0E0808181608083E1E9F0E08081826008
:103690008083808181608083E0E9F0E080818160C7
:1036A0008083E1ECF0E080818460808380818260AF
:1036B0008083808181608083E3ECF0E080818160A1
:1036C0008083E0ECF0E0808182608083E2ECF0E0D7
:1036D000808181608083EAE7F0E08081846080837C
:1036E0008081826080838081816080838081806826
:1036F0008083089590E0FC013197EE30F10590F55C
:10370000E35AFF4F0C941A26809180008F7703C0F4
:10371000809180008F7D80938000089584B58F779D
:1037200002C084B58F7D84BD0895809190008F770D
:1037300007C0809190008F7D03C080919000877FAB
:103740008093900008958091C0008F7703C080918E
:10375000C0008F7D8093C00008958091C200877F54
:103760008093C2000895CF93DF9390E0FC01E75E61
:10377000FE4F2491FC01E95CFE4F8491882349F1BE
:1037800090E0880F991FFC01EF58FE4FA591B4916E
:103790008D599E4FFC01C591D4919FB7611108C00E
:1037A000F8948C91209582238C93888182230AC07F
:1037B000623051F4F8948C91322F309583238C939E
:1037C0008881822B888304C0F8948C91822B8C93FF
:1037D0009FBFDF91CF910895A1E0B0E0E2EFFBE160
:1037E0000C94F125282F30E0F901E550FF4F84912A
:1037F000F901E75EFE4F1491F901E95CFE4F049177
:103800000023C9F0882321F069830E947A1B698113
:10381000E02FF0E0EE0FFF1FED59FE4FA591B491A0
:103820009FB7F8948C91611103C01095812301C05A
:10383000812B8C939FBF2196E4E00C940D26CF93AF
:10384000DF93282F30E0F901E550FF4F8491F90113
:10385000E75EFE4FD491F901E95CFE4FC491CC23A1
:1038600091F081110E947A1BEC2FF0E0EE0FFF1F08
:10387000EB5AFE4FA591B4912C912D2381E090E05D
:1038800021F480E002C080E090E0DF91CF910895C4
:10389000809154049091550420915604309157041E
:1038A000821B930B8F7399270895209154043091B4
:1038B000550480915604909157042817390749F010
:1038C000E0915604F0915704EC5EFB4F808190E04C
:1038D00008958FEF9FEF089520915404309155047F
:1038E000809156049091570428173907A9F0E09168
:1038F0005604F0915704EC5EFB4F808120915604F2
:10390000309157042F5F3F4F2F7333273093570465
:103910002093560490E008958FEF9FEF0895CF9382
:10392000DF93C0915404D09155042196CF73DD27C5
:103930008091560490915704C817D90799F082E0F6
:103940000E9444218F3F2FEF920761F0E0915404D1
:10395000F0915504EC5EFB4F8083D0935504C093E7
:103960005404DFCFDF91CF91089583E00E948F232D
:103970000895A1E0B0E0EFEBFCE10C94F1258C019F
:1039800069838091A401882359F041E050E0BE0191
:103990006F5F7F4F83E00E947721181619063CF075
:1039A00081E090E0F8019383828380E090E02196AB
:1039B000E4E00C940D26FC0120812E5F208342E47C
:1039C00050E06FE771E080E80E94F7210895FC0164
:1039D00081819081913A59F4813209F04BC047E0DE
:1039E00050E06DE971E080E00E94F72145C091321E
:1039F00009F040C0803239F467E070E08DE991E071
:103A00000E943B2239C0823209F034C08281809307
:103A1000A40180919D0190919E01A0919F01B09180
:103A2000A001803B9440A105B10531F58091A4012E
:103A300080FD12C087E797E7909301088093000804
:103A40002BE088E190E00FB6F894A8958093600091
:103A50000FBE2093600010C088E10FB6F8948093E9
:103A60006000109260000FBEA8951092010810929D
:103A7000000802C080E0089581E008950895109242
:103A800009041092080488EE93E0A0E0B0E080936F
:103A90000A0490930B04A0930C04B0930D048EE2DF
:103AA00092E090930704809306040895A0E0B0E0AC
:103AB000ECE5FDE10C94ED256C017A01EB01E60EDD
:103AC000F71E00E010E0CE15DF0561F06991D60128
:103AD000ED91FC910190F081E02DC6010995080F50
:103AE000191FF1CFC801CDB7DEB7E8E00C94092665
:103AF0006115710589F0DB010D900020E9F7AD013A
:103B000041505109461B570BDC01ED91FC9102809D
:103B1000F381E02D0995089580E090E00895EF92FB
:103B2000FF920F931F93CF93DF938C01FB01C0E0B3
:103B3000D0E064917F018FEFE81AF80A662361F004
:103B4000D801ED91FC910190F081E02DC80109951B
:103B5000C80FD91FF701EDCFCE01CDB7DEB7E6E034
:103B60000C940B260E94781D0895DC01ED91FC91C8
:103B70000190F081E02D099508950F931F93CF9345
:103B8000DF93EC016DE00E94B51D8C016AE0CE016F
:103B90000E94B51D800F911FDF91CF911F910F9152
:103BA00008950F931F93CF93DF93EC010E948F1D15
:103BB0008C01CE010E94BD1D800F911FDF91CF911E
:103BC0001F910F9108950F931F93CF93DF93EC01F3
:103BD0000E94781D8C01CE010E94BD1D800F911F97
:103BE000DF91CF911F910F9108950F931F93CF9362
:103BF000DF93EC010E94B51D8C01CE010E94BD1D1A
:103C0000800F911FDF91CF911F910F910895A1E235
:103C1000B0E0EDE0FEE10C94E9257C01C42EE52F37
:103C2000CB01D22E19A221E02D1510F02AE0D22EC0
:103C30008E010F5D1F4F8D2C912CA12CB12C6C2D62
:103C40007E2FA50194010E94A2258C2DD29E801961
:103C50001124015011098A3010F4805D01C0895C83
:103C6000F8018083211531054105510521F0C22E4F
:103C7000E32FCA01E4CFB801C7010E94781DA196C5
:103C8000ECE00C940526A0E0B0E0E9E4FEE10C9441
:103C9000ED25EC016A017B012115310541F4E88134
:103CA000F9810190F081E02D642F09951DC02A3023
:103CB0003105A9F477FF12C06DE20E94B51D8C0199
:103CC00044275527BA014C195D096E097F092AE07E
:103CD000CE010E94071E800F911F06C02AE0B70187
:103CE000A601CE010E94071ECDB7DEB7E8E00C9416
:103CF00009260F931F93CF93DF93EC019A01AB0139
:103D0000662757FD6095762F0E94431E8C01CE01D9
:103D10000E94BD1D800F911FDF91CF911F910F91C8
:103D200008952115310549F4DC01ED91FC910190D4
:103D3000F081E02D642F099508950E94071E0895D3
:103D40009A01462F50E060E070E00E94911E0895B5
:103D50009A01AB0160E070E00E94911E08950F93FC
:103D60001F93CF93DF93EC019A01462F50E060E060
:103D700070E00E94911E8C01CE010E94BD1D800F3B
:103D8000911FDF91CF911F910F910895FC01248520
:103D90003585F901E05CFF4F80819181F901EE5B8F
:103DA000FF4F20813181821B930B8F7399270895D8
:103DB000FC0184859585FC01E05CFF4F40815181C9
:103DC000FC01EE5BFF4F208131814217530741F028
:103DD0000190F081E02DE80FF91F808190E00895B7
:103DE0008FEF9FEF0895FC0184859585FC01E05CD1
:103DF000FF4F40815181FC01EE5BFF4F20813181FB
:103E00004217530779F0A081B181A80FB91F8C9197
:103E1000208131812F5F3F4F2F73332731832083E0
:103E200090E008958FEF9FEF0895FC0181A1882312
:103E300029F0A489B5898C9186FFFBCF11A2089542
:103E4000CF93DF93FC0126853785D901A05CBF4F56
:103E50008D919C91119701968F739927E901CE5B03
:103E6000DF4F4881598184179507D9F30D90BC9194
:103E7000A02DA20FB31F6C93A685B785A05CBF4F82
:103E800011969C938E93A689B7892C9181E090E03E
:103E9000078C02C0880F991F0A94E2F7282B2C93F5
:103EA00081E081A30488F589E02D8081806480838E
:103EB00081E090E0DF91CF91089508951F920F92D5
:103EC0000FB60F9211242F933F934F938F939F938D
:103ED000EF93FF938091C80082FD1CC04091CE00FB
:103EE0008091FE049091FF0401968F739927209191
:103EF0000005309101058217930771F0E091FE04EF
:103F0000F091FF04E254FB4F40839093FF048093B1
:103F1000FE0402C08091CE00FF91EF919F918F919E
:103F20004F913F912F910F900FBE0F901F901895BA
:103F300088E594E00E94C61E892B11F00E945D1F47
:103F400008951F920F920FB60F9211242F933F9353
:103F50008F939F93EF93FF932091BA043091BB040A
:103F60008091BC049091BD042817390731F48091E9
:103F7000C9008F7D8093C90014C0E091BC04F0910A
:103F8000BD04E658FB4F20818091BC049091BD0494
:103F900001968F7399279093BD048093BC0420935E
:103FA000CE00FF91EF919F918F913F912F910F90B4
:103FB0000FBE0F901F901895A0E0B0E0E2EEFFE179
:103FC0000C94E925FC011382128288EE93E0A0E0B4
:103FD000B0E084839583A683B78380E492E09183E5
:103FE00080837587648757874687318B208B138B37
:103FF000028BF58AE48AD78AC68AB18EA08E938E08
:10400000828E8F85848F8889858F8989868F8A891A
:10401000878F8B8980A3ECE00C940526CF92DF92EA
:10402000EF92FF92CF93DF93EC016A017B01411580
:1040300081EE580761057105F9F0EC89FD8981E091
:1040400090E008A002C0880F991F0A94E2F78083CD
:1040500060E079E08DE390E0A70196010E94A2253F
:1040600021503109410951095695479537952795B2
:10407000211580E1380798F0EC89FD89108260E80D
:1040800074E88EE190E0A70196010E94A2252150DC
:104090003109410951095695479537952795E88982
:1040A000F9893083EA89FB89208319A2EE89FF8987
:1040B000408181E090E09C010C8C02C0220F331FF4
:1040C0000A94E2F7422B4083EE89FF8940819C01EC
:1040D0000D8C02C0220F331F0A94E2F7422B40835B
:1040E000EE89FF8940819C010E8C02C0220F331F94
:1040F0000A94E2F7422B4083EE89FF8920810F8CDE
:1041000002C0880F991F0A94E2F78095822380836A
:10411000DF91CF91FF90EF90DF90CF9008958F9235
:104120009F92AF92BF92CF92DF92EF92FF920F9346
:104130001F9381E08F9385E08F9387E08F9383E0D7
:104140008F9384E08F93EEEC8E2E912CFAECAF2EB1
:10415000B12CA9ECCA2ED12CB8ECEB2EF12C0CEC26
:1041600010E02DEC30E04AE754E06EEB74E088E5B7
:1041700094E00E94DC1F0F900F900F900F900F9013
:104180001F910F91FF90EF90DF90CF90BF90AF9075
:104190009F908F9008950E94241B82E095E00E94DA
:1041A00099230E94DC14C8E9DFE10E947E17209762
:1041B000E1F30E94981FF9CF615030F02091F10097
:1041C000FC0120830196F8CF289884E680930905A6
:1041D00008952FB7FC012083F89467706093E9007D
:1041E0000895A1E0B0E0E7EFF0E20C94F325682F2A
:1041F000CE0101960E94E9208091F20099819FBF33
:104200002196E2E00C940F26A2E0B0E0EAE0F1E2B1
:104210000C94F025F62E8A0190910805992311F04F
:1042200057FF03C08FEF9FEF2BC0682FCE01019681
:104230007A830E94E9208091F20090E0A8017A81BF
:10424000801791070CF4AC01EF2DF72FF40E84E6E4
:10425000FE1639F02898809309059091F10091930A
:10426000F7CF4115510521F08091F200882321F00C
:1042700089818FBFCA0104C08BE68093E800F8CF24
:104280002296E5E00C940C26A1E0B0E0EAE4F1E22D
:104290000C94F32541E050E0BE016F5F7F4F0E9418
:1042A0000421019719F4898190E002C08FEF9FEFFC
:1042B0002196E2E00C940F26A1E0B0E0E2E6F1E204
:1042C0000C94F325682FCE0101960E94E92090916D
:1042D000E800892F807295FF04C09091F20080E47D
:1042E000891B99819FBF2196E2E00C940F26A1E0E3
:1042F000B0E0EDE7F1E20C94E525582E7B01A42E09
:10430000952E80910805882369F0042F152F8AEFD8
:10431000B82E852D8072782E9AE3892E852D807493
:10432000682E11C08FEF9FEF53C0852D0E945C2136
:10433000482E81110CC0BA94A9F361E070E080E0CE
:1043400090E00E94FE1A0115110579F737C0282F59
:1043500030E0021713070CF4402EC42CD12C0C199A
:104360001D09652DCE0101960E94E920772039F0C4
:104370004A948FEF4816B1F01092F100F9CFF7018F
:10438000842D57FE07C0815058F094919093F1000E
:104390003196F9CF815020F091919093F100FACFAE
:1043A000EC0CFD1C8091E80085FF0FC00115110584
:1043B00011F461100AC089818FBFC5CF5D9884E672
:1043C00080930A058A2D992D03C08092E800F3CFCF
:1043D0002196E0E10C9401261092E9001092070565
:1043E0001092060590930505809304050895CF93D8
:1043F000DF93FB0120E030E0DEEF24173507A1F169
:1044000087FF02C0C49101C0C081A0910605B09190
:1044100007056091040570910505A617B707B4F468
:104420009091E8009570E1F39091E80092FD1EC034
:10443000C093F10060910605709107056F5F7F4F93
:104440006F737727672B11F4D093E800609106050E
:10445000709107056F5F7F4F7093070560930605A6
:104460002F5F3F4F3196C9CFC90102C08FEF9FEF39
:10447000DF91CF910895A1E0B0E0E1E4F2E20C9485
:10448000F225162F2091E80022FFFCCF612F7983BF
:104490000E94DC208BEF8093E800812F7981972F99
:1044A0002196E3E00C940E26A1E0B0E0EAE5F2E20A
:1044B0000C94F3251982CE0101960E94DB1CCE01DB
:1044C00001960E943324898190E02196E2E00C94C9
:1044D0000F261F920F920FB60F921124EF92FF92A8
:1044E0000F931F932F933F934F935F936F937F93FC
:1044F0008F939F93AF93BF93EF93FF93CF93DF93EC
:10450000CDB7DEB76297DEBFCDBF1092E9008091D4
:10451000E80083FFE7C068E0CE010A960E94DC2035
:1045200082EF8093E8009A8597FF05C08091E800AC
:1045300080FFFCCF03C08EEF8093E800892F807648
:1045400009F0B5C08B85811105C01092F100109261
:10455000F100C1C0282F2D7F213009F4BCC0853067
:1045600049F48091E80080FFFCCF8C8580688093BF
:10457000E300B1C0863009F072C02D85E888F98863
:10458000223071F580E090E02A8B0E94EC210E949D
:10459000542299E08E010F5F1F4FF801392F1192BD
:1045A0003A95E9F799832A892A8391E09E8390E8D6
:1045B00098879AEF99872091060530910705275F24
:1045C0003F4F3C832B838D83C7010E94EC2149E040
:1045D00050E0B80180E00E94F7210E9454227BC085
:1045E000C7012A8B0E94EC212A89223241F482E2FF
:1045F00090E00E943F24892B09F06DC070C02130EB
:1046000069F488899989089711F4209303058091AA
:104610000305882389F066EC71E016C0233009F0A9
:104620005EC08C85882359F0823061F0813009F0BA
:1046300056C06AEE71E008C068ED71E005C064E242
:1046400072E002C062E072E06115710509F447C0D2
:10465000FB01449150E080E80E94F7213CC0873084
:1046600009F43DC0883021F481E08093F10033C02B
:10467000893089F5937099F5E2ECF1E081E021E071
:1046800096E38093E9002093EB0034913093EC00A3
:104690009093ED008F5F3196853099F78EE7809388
:1046A000EA001092EA008C858093080514C088897E
:1046B00099890E94EC218E85811105C0CE010A9650
:1046C0000E94E71C06C0823051F4CE010A960E9477
:1046D0006124882321F08EEF8093E80003C081E2FB
:1046E0008093EB0062960FB6F894DEBF0FBECDBF8D
:1046F000DF91CF91FF91EF91BF91AF919F918F91FA
:104700007F916F915F914F913F912F911F910F91E9
:10471000FF90EF900F900FBE0F901F901895809311
:10472000E9008091F200882319F08AE38093E80081
:1047300008951092080581E08093D70080EA809365
:10474000D80082E189BD09B400FEFDCF61E070E0D0
:1047500080E090E00E94FE1A80E98093D8008CE00F
:104760008093E2001092E000559A209A08951F92DB
:104770000F920FB60F9211242F933F934F935F9395
:104780006F937F938F939F93AF93BF93EF93FF9319
:104790008091E1001092E10083FF0FC01092E900C8
:1047A00091E09093EB001092EC0092E39093ED0077
:1047B0001092080598E09093F00082FF26C083E0F5
:1047C0000E948F2382E00E94F120882321F086E05E
:1047D00094E00E948F1C80910A05882339F0809113
:1047E0000A05815080930A05882369F080910905A4
:1047F000882359F080910905815080930905811122
:1048000004C0289A02C05D9AF1CFFF91EF91BF9149
:10481000AF919F918F917F916F915F914F913F9158
:104820002F910F900FBE0F901F901895FF920F932E
:104830001F93CF93DF93EC01F62EE881F98104807A
:10484000F581E02D09958C01E881F9810680F781D9
:10485000E02D6F2DCE010995C8019927CDB7DEB7A0
:10486000E5E00C940C26FC0120812F5F208349E1B8
:1048700050E068EA72E080E80E94F721089545E67A
:1048800050E061EC72E080E80E94F7210895A1E019
:10489000B0E0EDE4F4E20C94EF2589838B017A011A
:1048A00041E050E0BE016F5F7F4F84E00E947721BE
:1048B000A701B80184E40E9477212196E6E00C94D8
:1048C0000B26FC0191818081813A31F481E09130A5
:1048D00091F0933089F411C0813271F49B3021F44E
:1048E00082818093A60105C09A3031F48281809341
:1048F000A50181E00895089580E00895FC011082EB
:104900000895FC011382128220E532E03183208376
:10491000089548E050E082E00E9447240895CF9334
:10492000DF93DC01683818F0E8E7E60F25C0E62FD2
:10493000F0E067FF11C0E058F10981E090E001C0AC
:10494000880FEA95EAF714969C911497982B149681
:104950009C931497E0E010C0E85DFD4FE491EE23D6
:1049600009F440C0E7FF08C014968C911497826048
:1049700014968C931497EF7716968C9116978E1742
:1049800041F117968C9117978E1719F118968C9103
:1049900018978E17F1F019968C9119978E17C9F008
:1049A0001A968C911A978E17A1F01B968C911B97D3
:1049B0008E1779F080E090E0ED01C80FD91F2E81AD
:1049C000211102C0EE8305C0019686309105A1F742
:1049D00009C0BD016C5F7F4FCD010E94892481E039
:1049E00090E008C081E090E013969C938E9312971C
:1049F00080E090E0DF91CF910895683818F0E8E703
:104A0000E60F25C0E62FF0E067FF12C0E058F1097D
:104A100021E030E001C0220FEA95EAF72095DC01A1
:104A200014963C911497322314963C93E0E00FC007
:104A3000E85DFD4FE491EE2329F1E7FF08C0DC01BA
:104A400014962C9114972D7F14962C93EF7720E0D9
:104A500030E0EE2351F0DC01A20FB31F16964C910B
:104A600016974E1302C016961C922F5F3F4F2630AA
:104A7000310579F7BC016C5F7F4F0E94892481E08A
:104A800090E0089580E090E00895FC01168217827E
:104A900010861186128613861482BC016C5F7F4FCC
:104AA0000E948924089587E195E00E947E248BE08E
:104AB00095E00E9481240895A29FB001B39FC00198
:104AC000A39F700D811D1124911DB29F700D811D3A
:104AD0001124911D08950E945C25A59F900DB49FFF
:104AE000900DA49F800D911D11240895B7FF0C9483
:104AF0006B250E946B25821B930B0895DB018F931E
:104B00009F930E946B25BF91AF91A29F800D911D35
:104B1000A39F900DB29F900D1124089597FB072E2F
:104B200016F4009407D077FD09D00E94202607FCD8
:104B300005D03EF4909581959F4F089570956195AD
:104B40007F4F0895A1E21A2EAA1BBB1BFD010DC0C9
:104B5000AA1FBB1FEE1FFF1FA217B307E407F5072D
:104B600020F0A21BB30BE40BF50B661F771F881F09
:104B7000991F1A9469F760957095809590959B019F
:104B8000AC01BD01CF010895052E97FB1EF40094E2
:104B90000E94DB2557FD07D00E94A22507FC03D009
:104BA0004EF40C94DB2550954095309521953F4F60
:104BB0004F4F5F4F089590958095709561957F4F09
:104BC0008F4F9F4F08952F923F924F925F926F9217
:104BD0007F928F929F92AF92BF92CF92DF92EF928D
:104BE000FF920F931F93CF93DF93CDB7DEB7CA1B0E
:104BF000DB0B0FB6F894DEBF0FBECDBF09942A8839
:104C0000398848885F846E847D848C849B84AA84E0
:104C1000B984C884DF80EE80FD800C811B81AA816D
:104C2000B981CE0FD11D0FB6F894DEBF0FBECDBF38
:104C3000ED010895EE0FFF1F0590F491E02D09940A
:104C4000AA1BBB1B51E107C0AA1FBB1FA617B707B2
:104C500010F0A61BB70B881F991F5A95A9F78095CE
:104C60009095BC01CD0108958F929F92AF92BF9213
:104C7000CF92DF92EF92FF92CF93DF93EC016881A6
:104C800079818A819B81611571058105910521F4E6
:104C900064E279ED8BE597E02DE133EF41E050E000
:104CA0000E94C42549015A019B01AC01A7EAB1E465
:104CB0000E946B256B017C01ACEEB4EFA501940161
:104CC0000E947925C60ED71EE81EF91EF7FE06C003
:104CD00081E0C81AD108E10880E8F80AC882D982C0
:104CE000EA82FB82C701B6019F77DF91CF91FF90E7
:104CF000EF90DF90CF90BF90AF909F908F900895EE
:104D00000E943426089586E091E00E94342608959A
:104D10006093060170930701809308019093090145
:104D20000895F999FECF92BD81BDF89A992780B573
:104D30000895262FF999FECF1FBA92BD81BD20BDDF
:104D40000FB6F894FA9AF99A0FBE01960895F8945E
:024D5000FFCF93
:104D520000001805200001000000FF000200020010
:104D62000200020002000200020002000200020031
:104D7200020002000200020002000280250000057B
:104D8200400AA1204EA50020244EA52C2330C0129B
:104D920000001A400AA1204EA5001B1E27522C23F8
:104DA200308025000005400AA1204EA50020244E97
:104DB200A52C2330004B000006400AD0009D49007C
:104DC2007B289D492C233000E1000005400A450163
:104DD200D7DC03B81E0EBF00232E48E801008A402C
:104DE2000A6001555502AD1E20000023C800E100F3
:104DF2000000000000010154582074696D656F7550
:104E0200742100456E746572696E67206164617019
:104E120074697665206368616E6E656C2073656C7B
:104E2200656374696F6E2C207069636B696E673A93
:104E3200007363616E6E6572206D6F6465004F7002
:104E4200656E4C52536E67205458207374617274AD
:104E5200696E672000206F6E20485720006D6F64D6
:104E6200756C65206C6F636B65643F0000070B0C0B
:104E720010111500160A1322312900000000B91C76
:104E8200561D481C6C1C551CB51C8F1C00000000D4
:104E9200201F561DC61EF31ED81E151F000000003F
:0A4EA2001624561D8F24FD2445251B
:1070000055C000006EC000006CC000006AC00000E7
:1070100068C0000066C0000064C0000062C00000DC
:1070200060C000005EC00000F2C400005AC0000052
:1070300058C0000056C0000054C0000052C00000FC
:1070400050C0000078C000004CC000004AC00000E2
:1070500048C0000046C0000044C0000042C000001C
:1070600040C000003EC000003CC000003AC000002C
:1070700038C0000036C0000034C0000032C000003C
:1070800030C000002EC000002CC000002AC000004C
:1070900028C0000026C0000024C0000022C000005C
:1070A00020C000001EC000001CC0000011241FBE34
:1070B000CFEFDAE0DEBFCDBF11E0A0E0B1E0E2E368
:1070C000FFE702C005900D92A83AB107D9F711E089
:1070D000A8EAB1E001C01D92AE3BB107E1F78FD342
:1070E00026C78ECFF89410926F00109281001092F4
:1070F00085001092840081E085BF15BE47985D9A97
:10710000289A0C94000008952091B2013091B301A7
:107110002F5F3F4F3093B3012093B201932F37FF7E
:1071200003C08EEF831B982F990F921710F4479886
:107130000895479A08951F920F920FB60F92112447
:107140002F938F939F93EF93FF931092850010924C
:1071500084008091A8019091A901009741F00197C6
:107160009093A9018093A801892B09F45D9A8091DD
:10717000AA019091AB01009741F001979093AB0168
:107180008093AA01892B09F4289AE0E0F0E0859128
:1071900094918F5F9F4F49F08091AC019091AD0128
:1071A00001969093AD018093AC01FF91EF919F9177
:1071B0008F912F910F900FBE0F901F90189584E024
:1071C0008093E9000DC08091E8008B778093E80000
:1071D00003C08EB3882351F08091E80082FFF9CF7D
:1071E0008091E80085FFEFCF8091F1000895982FFE
:1071F00083E08093E9008091E80085FD0DC08091D7
:10720000E8008E778093E80003C08EB3882369F08E
:107210008091E80080FFF9CF9093F1005D9884E6BB
:1072200090E09093A9018093A80108954F925F92F6
:107230006F927F928F929F92AF92BF92CF92DF9286
:10724000EF92FF920F931F93CF93DF9384E080938D
:10725000E9008091E80082FF57C2289884E690E018
:107260009093AB018093AA01AADF182F853481F493
:107270008CE49DE19093AD018093AC0107B600FCD6
:10728000FDCFF999FECF81E180935700E89503C0C7
:10729000843519F494DF8DE00DC28C34E1F3803530
:1072A000D1F3843721F484E4A2DF80E003C2813685
:1072B00011F489E5FFC18134B1F481DF182F7FDF3C
:1072C00090E0880F991FAA2797FDA095BA2F312F1C
:1072D000330F20E0442737FD4095542F822B932B0A
:1072E000A42BB52BB8C1803711F483E5E3C18335F6
:1072F00049F4C0E0D1E089917ADF21E0C730D207BC
:10730000D1F7D9C1863521F481E371DF80E3D2C1A1
:10731000833731F487E86BDF85E969DF8EE1CAC125
:107320008536B9F4E0E0F0E093E085E09093570013
:10733000E89507B600FCFDCF80935700E89507B6A7
:1073400000FCFDCFE058FF4FA0E7E030FA0771F7EF
:10735000A2CF823739F4E1E0F0E089E08093570072
:107360008491A8C1863439F4E0E0F0E089E08093AC
:10737000570084919FC18E3439F4E3E0F0E089E056
:1073800080935700849196C1813539F4E2E0F0E0B2
:1073900089E08093570084918DC1823631F489E56C
:1073A00026DF80E024DF80E885C1823419F087364B
:1073B00009F0E5C01092AD011092AC0100DF082F7A
:1073C000FEDEF82EFCDE682E8554823008F071C196
:1073D000902F80E0CF2DD0E0C82BD92B10926F00DA
:1073E000173609F04BC081E180935700E895DD2402
:1073F000CC24C3943FC0E090AE01F090AF01009167
:10740000B0011091B101B6E46B16D9F4ED2DF0E0A6
:10741000EE29FF29E4918E2FEADEDD2081F082E063
:1074200090E0A0E0B0E0E80EF91E0A1F1B1FE092FA
:10743000AE01F092AF010093B0011093B101DC24D2
:1074400018C0D801C701B695A7959795879559D5C6
:10745000CEDE82E090E0A0E0B0E0E80EF91E0A1F68
:107460001B1FE092AE01F092AF010093B0011093A8
:10747000B1012197209709F0BECF7DC08090AE0169
:107480009090AF01A090B001B090B10196E4691660
:1074900009F05DC083E0F40180935700E89507B6DA
:1074A00000FCFDCF54C0F6E46F1661F5772031F192
:1074B000E090AE01F090AF010091B0011091B101E8
:1074C0007EDED82ECC24852D90E08C299D29F701D5
:1074D0000C0140925700E895112482E090E0A0E072
:1074E000B0E0E80EF91E0A1F1B1FE092AE01F092F9
:1074F000AF010093B0011093B10102C060DE582EBD
:10750000742423C0E090AE01F090AF010091B0016F
:107510001091B10116950795F794E79450DE682F06
:10752000C701F7D48091AE019091AF01A091B00155
:10753000B091B1010296A11DB11D8093AE0190934F
:10754000AF01A093B001B093B101219704C05524BD
:10755000772444244394209709F0A5CF96E4691634
:1075600041F485E0F40180935700E89507B600FCEC
:10757000FDCF8DE03CDE82E080936F009CC08334C1
:1075800071F40091AE011091AF0119DE90E021E09D
:10759000F8010C0120935700E89511247CCE833626
:1075A00019F5E090AE01F090AF010091B00110919B
:1075B000B10105DEF701E16090E021E00C012093CC
:1075C0005700E895112482E090E0A0E0B0E0E80EDA
:1075D000F91E0A1F1B1FE092AE01F092AF0100934B
:1075E000B0011093B10157CE8D3661F4E091AE0138
:1075F000F091AF0185E080935700E89507B600FC55
:10760000FDCF49CE823551F4E091AE01F091AF014A
:1076100005911491812FEBDD802F4CC0843421F52E
:10762000E090AE01F090AF010091B0011091B10176
:1076300016950795F794E794C2DD682FC70169D4C2
:107640008091AE019091AF01A091B001B091B101D4
:107650000296A11DB11D8093AE019093AF01A0933E
:10766000B001B093B10117CE843609F5E090AE01B8
:10767000F090AF010091B0011091B101D801C701A4
:10768000B695A795979587953CD4B1DD82E090E0BB
:10769000A0E0B0E0E80EF91E0A1F1B1FE092AE0149
:1076A000F092AF010093B0011093B10104C08B318F
:1076B00011F08FE39CDD83E08093E9009091E80076
:1076C0008091E8008E778093E80095FF04C010C099
:1076D0008EB38823C9F08091E80080FFF9CF8091B4
:1076E000E8008E778093E80003C08EB3882361F0B2
:1076F0008091E80080FFF9CF84E08093E9008091D9
:10770000E8008B778093E800DF91CF911F910F9174
:10771000FF90EF90DF90CF90BF90AF909F908F90B1
:107720007F906F905F904F9008959091B601892F50
:107730008F77813249F58091B7018032A1F0813293
:1077400019F5913A09F58091E800877F8093E80068
:107750008DE091E067E070E00BD28091E8008B77DC
:107760008093E8000895913279F48091E800877F52
:107770008093E8008DE091E067E070E05DD2809159
:10778000E8008E778093E800089582E061EC42E0A3
:10779000B5D083E061E842E1B1D084E060E842E145
:1077A000ADC084B7877F84BF88E10FB6F89480931B
:1077B0006000109260000FBE20E880E090E00FB6FD
:1077C000F89420936100809361000FBE81E085BF33
:1077D00092E095BF3F9A209A559AE1E6F0E0208327
:1077E000108247985D9A289A109289008AEF8093B8
:1077F000880090936F0083E080938100F0C04091F7
:10780000000850910108109201081092000894B7E6
:1078100014BE88E10FB6F894809360001092600067
:107820000FBE292F30E0F901E270F07091FD18C011
:1078300090FF05C0859194918F5F9F4F81F423FF46
:107840000FC08091090190910A014817590741F032
:10785000E0E0F0E0859194918F5F9F4F09F042DC6A
:10786000A0DF78941092AD011092AC010CC0DEDC68
:1078700036D38091AC019091AD0181549F4110F0BD
:107880001092140141DC80911401882381F78091CA
:10789000E00081608093E00025DC80E090E00895C6
:1078A000FA01923049F0933061F09130F9F485E1BA
:1078B00091E022E130E01EC087E291E02EE330E06B
:1078C00019C0882329F485E691E024E030E012C055
:1078D000813029F489E691E022E230E00BC0823069
:1078E00029F48DE891E028E130E004C080E090E0E8
:1078F00020E030E091838083C90108958093E900FE
:107900008091EB0081608093EB001092ED0060931A
:10791000EC004093ED008091EE00881F8827881FBF
:1079200008958091B60188238CF403C08EB3882318
:10793000B1F08091E80082FFF9CF8091E8008B7769
:107940008093E80008958EB3882349F08091E80081
:1079500080FFF9CF8091E8008E778093E80008954A
:10796000EF92FF920F931F9345D04CD008ED10E09B
:10797000F80180818F778083808180688083808117
:107980008F7D808319BC1EBA1092B40180EEE82E60
:10799000F12CF70180818B7F8083F80180818160E9
:1079A000808380E060E042E0A9DFE1EEF0E08081EA
:1079B0008E7F8083E2EEF0E0808181608083808131
:1079C00088608083F70180818E7F8083F8018081C9
:1079D000806180831F910F91FF90EF900895E7EDF4
:1079E000F0E08081816080838AE482BF81E08093BF
:1079F000B501B6CFE8EDF0E080818E7F80831092F4
:107A0000E20008951092DA001092E10008951F92AA
:107A10000F920FB60F9211242F933F934F935F93C2
:107A20006F937F938F939F93AF93BF93EF93FF9346
:107A30008091DA0080FF1BC08091D80080FF17C0C2
:107A40008091DA008E7F8093DA008091D90080FFE8
:107A50000BC080E189BD82E189BD09B400FEFDCF84
:107A600081E08EBB3BD203C019BC1EBA37D28091D5
:107A7000E10080FF17C08091E20080FF13C0809179
:107A8000E2008E7F8093E2008091E200806180932B
:107A9000E2008091D80080628093D80019BC85E014
:107AA0008EBB1CD28091E10084FF2CC08091E2004B
:107AB00084FF28C080E189BD82E189BD09B400FE50
:107AC000FDCF8091D8008F7D8093D8008091E10018
:107AD0008F7E8093E1008091E2008F7E8093E200B0
:107AE0008091E20081608093E2008091B40188235C
:107AF00031F48091E30087FD02C081E001C084E0A1
:107B00008EBBECD18091E10083FF21C08091E20027
:107B100083FF1DC08091E100877F8093E10082E0B8
:107B20008EBB1092B4018091E1008E7F8093E100C2
:107B30008091E2008E7F8093E2008091E20080617C
:107B40008093E20080E060E042E0D8DEC7D1FF91A0
:107B5000EF91BF91AF919F918F917F916F915F91C5
:107B60004F913F912F910F900FBE0F901F9018953E
:107B70009C014091BC015091BD014617570718F474
:107B8000F90190E044C06115710511F0AB01F8CF27
:107B90008091E8008E778093E80040E050E0F0CFDD
:107BA0008EB3882309F444C0853009F443C0809122
:107BB000E80083FF02C081E008958091E80082FD23
:107BC00031C08091E80080FF22C08091F300909145
:107BD000F200782F60E0292F30E0262B372B07C0EA
:107BE00081918093F100415050402F5F3F4F4115EC
:107BF000510519F02830310598F390E0283031050F
:107C000009F491E08091E8008E778093E8004115B7
:107C1000510531F6992321F605C08EB3882341F032
:107C2000853041F08091E80082FFF7CF80E0089531
:107C300082E0089583E008959C016115710529F49F
:107C40008091E8008B778093E800F90126C08EB31D
:107C5000882391F1853091F18091E80083FF02C083
:107C600081E008958091E80082FFF1CF06C0809105
:107C7000F10081936150704059F02091F3008091A0
:107C8000F200322F20E090E0822B932B892B79F7A2
:107C90008091E8008B778093E80061157105B9F653
:107CA00005C08EB3882341F0853041F08091E80013
:107CB00080FFF7CF80E0089582E0089583E0089583
:107CC0000F931F93DF93CF9300D0CDB7DEB7E6EBD2
:107CD000F1E08091F100819381E0EE3BF807C9F774
:107CE00024DD8091E80083FFE4C08091B60190918B
:107CF000B701953009F46DC0963040F4913081F1B0
:107D0000913070F0933009F0D4C02AC0983009F453
:107D1000A3C0993009F4B2C0963009F0CAC07CC043
:107D2000803809F4C6C0823809F0C3C08091BA0116
:107D300087708093E9008091EB001092E900209118
:107D4000E800277F2093E80090E025E0969587954E
:107D50002A95E1F781708093F1001092F10087C0BD
:107D6000882319F0823009F0A4C08F71823009F0A5
:107D7000A0C08091B801882331F52091BA01277005
:107D800009F497C02093E9008091EB0080FF1BC0AD
:107D9000933021F48091EB00806213C08091EB005E
:107DA00080618093EB0081E090E002C0880F991F12
:107DB0002A95E2F78093EA001092EA008091EB00A6
:107DC00088608093EB001092E9008091E800877F43
:107DD00051C0882309F06DC01091B8011F770FB70B
:107DE000F8948091E800877F8093E8009ADD809185
:107DF000E80080FFFCCF8091E3008078812B8093A6
:107E0000E30080688093E300112311F482E001C055
:107E100083E08EBB0FBF4DC08058823008F049C050
:107E20008091B8019091B9016091BA01AE014F5FA4
:107E30005F4F36DDBC01009709F43BC08091E8003C
:107E4000877F8093E80089819A8192DE8091E800A3
:107E50008B778093E8002DC0803859F58091E80039
:107E6000877F8093E8008091B4018093F100809136
:107E7000E8008E778093E80054DD1BC08823C9F4A6
:107E80009091B8019230A8F48091E800877F8093A8
:107E9000E8009093B40145DD8091B401882331F46A
:107EA0008091E30087FD02C081E001C084E08EBBC9
:107EB0006CDC8091E80083FF0AC08091EB00806257
:107EC0008093EB008091E800877F8093E8000F901B
:107ED0000F90CF91DF911F910F91089508951F93F7
:107EE0008EB3882361F01091E9001092E90080912F
:107EF000E80083FF01C0E4DE17701093E9001F91D2
:107F00000895F999FECF92BD81BDF89A992780B561
:107F10000895262FF999FECF1FBA92BD81BD20BDCD
:107F20000FB6F894FA9AF99A0FBE01960895F8944C
:107F3000FFCF4341544552494E4100777700080036
:107F400000000000000801120110010200000841B9
:107F500023360001000201000109023E0002010077
:107F60008032090400000102020100052400100112
:107F7000042402040524060001070582030800FF0B
:107F800009040100020A00000007050402100001B4
:107F90000705830210000104030904220341007253
:107FA000006400750069006E006F0020004C0065E1
:107FB000006F006E006100720064006F0000001826
:107FC00003410072006400750069006E006F0020BC
:0A7FD000004C004C004300000000CC
:00000001FF
